:10000000020385020A71FFFFFFFFFF020A83FFFF61
:10001000FFFFFF020A7BFFFFFFFFFF020B6FFFFFE7
:10002000FFFFFFFFFFFFFFFFFFFFFFFFFFFFFFFFE0
:10003000FFFFFFFFFFFFFFFFFFFFFFFFFFFFFFFFD0
:10004000FFFFFF020385C29075831E758200D58273
:10005000FDD583FA74201200FC74801200FC7583B5
:100060000F758200D582FDD583FA74201200FC74CE
:10007000801200FC758301758233D582FDD583FA29
:100080007406120095740C120095741412009522D7
:10009000D290C29022C0E01200CAC0E054F0120018
:1000A000FCD0E0C454F01200FCD0E022C0E07401A7
:1000B00080E5C0E0740280DFC0E0748080D9C0E0D9
:1000C00074C080D3C0E0448080CDC0E05390FA4338
:1000D00090F2D290E590C290D290C29020E7F3D0F7
:1000E000E022C0E011CAC0E054F044041200FCD089
:1000F000E0C454F044041200FCD0E02244085290C2
:1001000054F74290808AC0E0742080D811B8C0E0D3
:100110001581D083D082058105810581740093B457
:100120000010A3158115811581C082C0830581D07F
:10013000E022B41F00400211E2B40206A37400934F
:1001400011C4A380D711BE80C5540F04832230315F
:1001500032333435363738394142434445463149E4
:1001600011E222C0D0C0E0C4315ED0E0315ED0D018
:100170002240028009C0E0743111E2D0E022C0E0E8
:10018000743080F5758300858382780AD582FDD529
:1001900083FAD8F82211461146114611461146112C
:1001A000AC22C083C082858325858226D082D083FD
:1001B00022C0E053D0FF43D01831A2F5271201DA54
:1001C0001201C953D0E7D0E02253D0FF43D01831F9
:1001D000A2120298E52753D0E72212023574057F58
:1001E00004120229E5257F0312022974007F0112FF
:1001F0000229120257E5267F08120229120257E54A
:10020000277F0812022912025712024812021022F6
:100210007B40DB02800F12023574857F08120229B1
:1002200012025740ED12024822C2A1C2A11392A0AD
:10023000D2A1DFF7220000D2A10000D2A00000C2AC
:10024000A00000C2A10000220000C2A00000D2A1B4
:100250000000D2A000002200000000C2A10000D2D5
:10026000A000000000D2A1000000000000A2A0C277
:10027000A10000220000C2A10000C2A000000000F6
:10028000D2A10000C2A10000D2A0000022D2A00092
:1002900000D2A10000C2A122513574057F0451296A
:1002A000E5257F03512974007F0151295157E52627
:1002B0007F0851295157513574057F045129E5258F
:1002C0007F03512974017F01512951577F08D2A121
:1002D0000000A2A0C2A1E52713F527DFF1518D513F
:1002E0004851482230010312098FE5A054F0300133
:1002F0000C12098F12098F12098F12098FB4F004A2
:10030000743FC322E5A054F064F060D864F0C49058
:100310000315938010000C0B0906040E0A050D0846
:10032000030702010FD32251E450FCC083C0827541
:100330008308758200D582FDD583FAD082D083519F
:10034000E450E4C0E051E440FCD0E022744A11C41F
:10035000747F11E2747E11E2747811E274DA11E2B2
:1003600022744A11C474DA11E211E211E211E2229C
:10037000744A11C4747F11E2747E11E2742F11E289
:1003800074DA11E222121BEF7800E4F608B880FB61
:1003900075A80075D00075817F3195310E02044437
:1003A0004453202056464F00120A2E3184318411C6
:1003B000AC310E020B56332E313600318411AC12A3
:1003C0001E37754E18C201C203C202C200C20E51CE
:1003D000E4B40321310E0201726573657400712764
:1003E000310E02403E0090000074FF31B1A3E5835E
:1003F000B408F611AC12168B200117E5587004D220
:100400000A8002C20AE5577002D293E548600312DF
:1004100018DA51E4200A030208EA20020F2001063C
:10042000201C0602042F0205A40207BB020834B4F4
:100430000106120CE40208EAB402061212270208AE
:10044000EAB403061212F90208EAB40411310E02EA
:100450000D6C736200C284D28571270208EAB4056C
:1004600011310E020D75736200C285D284712702AC
:1004700008EAB4061A310E020D6377200020230625
:10048000D284D2858004B285B28471270208EAB48E
:100490000720310E020D3C3C3C0071271218B515A7
:1004A00052E552B4FF0375520A120A13120A1F02D0
:1004B00008EAB4081F310E020D43525300C20FC2A6
:1004C0000D200006D200D20C8002C2007127121546
:1004D0002B0208EAB40920310E020D3E3E3E0071A7
:1004E000271218B50552E552B40B03755200120AD3
:1004F00013120A1F0208EAB40A061214420208EA9A
:10050000B40B10310E020D66736B001210137127BD
:100510000208EAB40C25310E020D747868007127C8
:10052000310E020D54784800E551C0E07551037456
:1005300004121507D0E0F5510208EAB40D1D310E82
:10054000020D524954007127E551C0E07551037402
:10055000031214F0D0E0F5510208EAB40E1D310E7A
:10056000020D53504C007127E551C0E075510374E2
:10057000021214E7D0E0F5510208EAB4002330205B
:1005800017310E020D423A2000D201D20285A82A6C
:1005900075A884712702098685A82A75A88402088F
:1005A000370208EAF529B4010C1207B4743111E2DC
:1005B00071270206DFB4020C1207B4743211E27123
:1005C000270206DFB4030C1207B4743311E271275B
:1005D0000206DFB4040C1207B4743411E27127026E
:1005E00006DFB4050C1207B4743511E27127020658
:1005F000DFB4060C1207B4743611E271270206DF6D
:10060000B4070C1207B4743711E271270206DFB485
:10061000080C1207B4743811E271270206DFB4091E
:100620000C1207B4743911E271270206DFB40A43D1
:10063000310E020D463E4100300308310E020D46D8
:100640003E3E0071271207AA200D03300003300C34
:100650000312073FC201786E7937300302795E12C8
:100660001A69852AA830030511AC020C01120A1F71
:100670000208EAB40B2E2003C2310E020D463E42A0
:100680000071271207AA200D03300003200C03126B
:10069000073FC201786E793B121A69120A1F852A38
:1006A000A80208EAB40C1A310E020D45534300713A
:1006B000271207AAC201852AA82003AC11AC0208A0
:1006C000EAB40D0280E1B40E0280DCB4000B120724
:1006D000B4743011E271278006B43F03020986E545
:1006E00029C3AF28BF0303C4F56EBF0407426EE5FC
:1006F0006E120764BF0603C4F56FBF0702426FBFE7
:100700000803C4F570BF0A084270200303301C0BB5
:10071000BF0B03C4F571BF0C0F4271752800200395
:1007200005200C02C183C145BF04071207B474053C
:1007300011C4BF08071207B4740911C40209862046
:100740001C2120031E301D1BE553B4FF0A310E028D
:100750004D4F757400C1A71218B5855352120A1374
:10076000120A1F227553FFB40103755300B403032B
:10077000755301B40703755302B41003755303B4E2
:100780001403755304B41803755305B4210375534A
:1007900006B42403755307B42803755308B45003F3
:1007A000755309B4440375530A22740C11952274CD
:1007B0000F119522E528052811C422B4010302086F
:1007C000EAB40206120B950208EAB403061212F903
:1007D0000208EAB4071A310E024D3E443200712776
:1007E000D226121A61121C2B121B98C2260208EA8A
:1007F000B40810310E020D4F4646007127121C0E30
:100800000208EAB4091F12010E020D3E4432001222
:1008100003271200ACD226121A5D121C2B121B9851
:10082000C2260208EAB40A030204F7B40003020570
:100830007B0208EAB4005B12010E020C2046525102
:1008400000C202D201752802756E00756F007570C6
:10085000007571001203271207AF1200AC12010ECF
:100860000200463D0012010E02042C0012010E028D
:10087000082E0020030B201C0812010E020A303043
:100880000012010E020D4D487A0074021200C402DB
:100890000986B43F0A12010E020F3F00020986B416
:1008A0000D028003B40E1712010E020F580012033E
:1008B00027C201C202852AA81200AC0208EA15E08C
:1008C000F553740F1200C47431255312015E1203E4
:1008D000271218B5855352120A13120A1FC201C2F9
:1008E00002852AA81200AC0208EA120A96301C03FC
:1008F000020979301E0F20A3061209990209791204
:1009000009EF020979200B1230A20530A3028005FD
:1009100012099980641209EF805F120A5230101A8E
:10092000120999C212120A5D120A0B120A5D85564B
:1009300058855557D28CD28EC210120A52301136B9
:10094000120999C212E577B40402D212120A5DB4F8
:100950000302D212120A5DB40202D212120A5DB46C
:100960000102D212120A0B120A5D8556588555579C
:10097000D28CD28EC2111209EF300A10121C6F12E3
:100980001CD0C28CC28E4387014387200203F8909B
:100990000555D582FDD583FA22300D08200E05D2EB
:1009A0000E12153D301E2F308609C286C293C20A30
:1009B000121B9820A210201F2975540520220375B0
:1009C0005403D21F8013301F19755403202203755E
:1009D0005405C21F8003308609C286C293C20A1220
:1009E0001B98855658855557D28CD28ED207223007
:1009F0000D11300E0E30930BC20EB20C12153DB21B
:100A00000CC20ED286121B0DC20722D286121B9870
:100A1000C20722E5529007FF1201B11215C122D27E
:100A200021121B0D1200AC121C6F121CD022744735
:100A30001200C474531200E294031200E2941D12D7
:100A400000E224201200E224041200E2940D1200BD
:100A5000E22220A202D21020A302D2112253A8FB2C
:100A6000AA7630120251527BFFDBFEDAF543A8046E
:100A70002230B4040548800215483232758CD8758E
:100A80008AF022C0E0517CE55860021558E55760B5
:100A9000021557D0E032E5805430B578028007D295
:100AA00021F578121B0D302003020AFBE580540F5C
:100AB000B552028046B40F1B1200ACE580540FB44F
:100AC0000F1112010E0201526561642042414E4431
:100AD0000080E81200AC7F007E00DEFEDFFAE580D9
:100AE000540FB5520280141218B5F5521215C112E6
:100AF0001B0D1200AC121C6F121CD0744E1200C4DD
:100B0000742020930474548005200A02744C02005F
:100B1000E2FB1DFC17FCBEFD35FD8EFDD4FE06C0BC
:100B200083C082C0E0E554B40005900B118030B45E
:100B30000105900B138028B40205900B158020B49A
:100B40000305900B178018B40405900B198010B49E
:100B50000505900B1B8008B40605900B1D8000E472
:100B600093F58D740193F58BD0E0D082D08322C0B1
:100B7000E0711F300704B2878004D287C28ED0E0B4
:100B800032E54820E7070303543FC38007F404031A
:100B900003543FD3221200AC12010E0200537465BD
:100BA000703A00C0E0E54DB4000F754D03C2091264
:100BB000010E02053130008032B4030F754D09C2B9
:100BC0000912010E0205316B008020B40911754D28
:100BD0000AC20912010E02053130306B00800C751B
:100BE0004D00C20912010E02053100D0E0020327B8
:100BF0001200AC12010E0200572073746570008061
:100C00000012010E0249487A207678745400120CC2
:100C10009E120C80200306301C03120327C203E53A
:100C200048603AC0E07548007563007564007565FA
:100C3000011202E4B40A0975630175640075650068
:100C4000B4030975630075640175650078617965A1
:100C5000D0E020E705121DE88003121DF4120C807D
:100C60001202E4C227B40207120CABD227800BB4E5
:100C70000005D203020598B401A3754800020327BA
:100C800074401200C47F04785EBF030A74421200ED
:100C9000C4742C1200E2E612016308DFEC227562D4
:100CA0000075630075640075650022755E00755FF0
:100CB000007560007561002212010E020220494693
:100CC00020002212010E020242414E440022120173
:100CD0000E020220534554002212010E0202204B44
:100CE00045590022C2081200ACE54EB4000A91B882
:100CF00012010E0207435700B4010B91B812010E06
:100D000002074C534200B4020B91B812010E0207C5
:100D100055534200B4030C91B812010E02074D4F17
:100D2000444500B4040C91CE12010E02074C4F430F
:100D30004B00B4050C91CE12010E0207484F4C44F3
:100D400000B4060C91D912010E020743484152002B
:100D5000B4071B91D9200B0C12010E0207454C451C
:100D60004300800A12010E02074E4F524D00B40894
:100D70000B91D912010E02074D454D00B4091B918C
:100D8000B820040C12010E020743573D3000800AC0
:100D900012010E020743572B2D00B40A1B91C320EA
:100DA0001D0C12010E02075741524300800A120126
:100DB0000E02075749444500B40B1F12010E0202F0
:100DC00046534B00201E0A12010E02074F4E0080B0
:100DD0000912010E02074F464600B40C1E91C320B3
:100DE000200F12010E0207535445520043800F801A
:100DF0000A12010E02075245414400B40D0C91C382
:100E000012010E02073136306D00B40E0B91C31281
:100E1000010E020738306D00B40F0B91C312010EA2
:100E2000020734306D00B4100B91C312010E02079B
:100E300033306D00B4110B91C312010E0207323032
:100E40006D00B4120B91C312010E020731376D0011
:100E5000B4130B91C312010E020731356D00B414A7
:100E60000B91C312010E020731326D00B4150B91C4
:100E7000C312010E020731306D00B4160B91C3127C
:100E8000010E020720366D00B4170B91C312010E3C
:100E9000020720326D00B4180A12010E02074558ED
:100EA00049540071816034D2087548004016054EDF
:100EB000E54E202007B40D047418F54EB4190375DF
:100EC0004E008014154EE54E202007B41704740C14
:100ED000F54EB4FF03754E181200AC1202E4500236
:100EE00081E9200800E54EB4001890000B785E12EE
:100EF00018AA910120270890000B785E12189F0213
:100F0000100EB4011890000F785E1218AA910120FB
:100F1000270890000F785E12189F02100EB4021876
:100F2000900013785E1218AA9101202708900013F0
:100F3000785E12189F02100EB403061210260210DB
:100F40000EB4040DE55612117EF55612185A021011
:100F50000EB4050DE55512117EF55512186B0210F1
:100F60000EB4060FE576F4121168F4F576121849FE
:100F700002100EB40715B20B9000071201C9A20BA4
:100F800092E79000071201B102100EB40810E57745
:100F90001211CCF5779000061201B102100EB409BF
:100FA00015B2049000071201C9A20492E69000074E
:100FB0001201B102100EB40A15B21D900007120101
:100FC000C9A21D92E59000071201B102100EB40BE8
:100FD0000612101302100EB40C1AB2209000071261
:100FE00001C9A22092E49000071201B1202003431E
:100FF000800F801AB418028015C0E01218B5D0E036
:10100000C3940DF5529007FF1201B11215C1D22100
:1010100002152BB21E201E081217A375540380025E
:10102000C20B1217F722755E401200AC900002123C
:1010300001C9F55AA31201C9F55B120370740012BD
:1010400000C4E55AA2E7120171A2E6120171A2E5FD
:10105000120171A2E4120171A2E3120171A2E21263
:101060000171A2E1120171A2E0120171E55BA2E738
:10107000120171E55E1200C474231200E21202E450
:10108000400302112D120327B4010A155EE55EB478
:101090003F03755E48B4020A055EE55EB449037518
:1010A0005E40B40370E55EB44009E55AB2E7F55A14
:1010B00002112AB44109E55AB2E6F55A02112AB4DE
:1010C0004209E55AB2E5F55A02112AB44309E55A34
:1010D000B2E4F55A02112AB44409E55AB2E3F55ACA
:1010E00002112AB44509E55AB2E2F55A02112AB4AE
:1010F0004609E55AB2E1F55A02112AB44709E55A00
:10110000B2E0F55A02112AB44809E55BB2E7F55B93
:1011100002112A8018B40A12900002E55A1201B195
:10112000900003E55B1201B180051200AC013AE5C5
:101130005AA2E79213A2E69214A2E59215A2E492B3
:1011400016A2E39217A2E29218A2E19219A2E092EB
:101150001AE55BA2E7921B229000021201C9F55A20
:10116000A31201C9F55B80C7F55E7548001200AC9B
:1011700012010E020073706565643A00801CF55E12
:101180007548001200AC12010E020054696D6572C0
:101190003A2020202030206D7300120361E55E129A
:1011A00019C474061200C4E55AC2281219D51202D5
:1011B000E44011E548600BF5F0E55E25F0F55E755D
:1011C000480080D61202E440FBE55E22F55E7548D9
:1011D000001200AC12010E02004D454D3A00120300
:1011E00061E55E1219C4740A1200C4E55AC22812DD
:1011F00019D51202E44020E548601A20E70AE55EAE
:1012000004B4050274008008E55E14B4FF0274049F
:10121000F55E75480080C71202E440FBE55E2212CD
:10122000010E020C530022C208E54FB4000B511FFF
:1012300012010E020D20203100B4010B511F1201CA
:101240000E020D20203200B4020B511F12010E02BB
:101250000D20203500B4030B511F12010E020D208A
:10126000313000B4040B511F12010E020D20323038
:1012700000B4050B511F12010E020D20353000B4D1
:10128000060B511F12010E020D31303000120B817E
:10129000601DD208754800400C054FE54FB40703A8
:1012A000754F00800A154FE54FB4FF03754F0612C6
:1012B00002E450024129200813E54D2009042403CB
:1012C0008003C39403B209F54D0212D6E54F854F52
:1012D0004D121841C20902152B12010E020C204DAD
:1012E000001213531201C904B40A027400C0E0745E
:1012F0000E1200C4D0E0020163755000E550B40046
:101300000451D98012B40B0C12010E020C2045536B
:10131000430080031213C5120B81601B7548004007
:101320000C0550E550B40C03755000800A1550E5CB
:1013300050B4FF0375500B1202E4500280BEE5501A
:10134000B400051213A58008B40B02800312140325
:1013500002152BC0E0301C06C21D74038008E55244
:10136000B40003900083B401039000DFB402039043
:10137000013BB40303900197B404039001F3B40557
:101380000390024FB406039002ABB4070390030727
:10139000B40803900363B409039003BFB40A039035
:1013A000041BD0E02271531201C904B40A004002A8
:1013B00074001201B112143278377E08E61201B1BE
:1013C00008A3DEF822C0E014C0E012010E020C20D7
:1013D0005200D0E0C0E0120163D0E0715312143229
:1013E0007E08785E1201C9F608A3DEF874021200C6
:1013F000C4785E121CA674421200C47862121CA645
:10140000D0E022147153121432785A7E081201C9A6
:10141000F608A3DEF8785D301D0C121A44401278ED
:101420005D121A2C400B785A79377F08121A6BC25A
:101430000F2275F009A4A32582F582E5F03583F526
:101440008322C208301E0F20080C12010E020D4626
:101450005352000214A0E551B4000912010E020D0E
:10146000412F4200B4010912010E020D413D42001C
:10147000B4020912010E020D53504C00B4030912BC
:10148000010E020D52495400B4040912010E020D5E
:1014900054784800B4050912010E020D4E4F500059
:1014A000120B81601DD208754800400C0551E551B2
:1014B000B40603755100800A1551E551B4FF037558
:1014C00051051202E450028144301E08200805B282
:1014D0002202152BE551B40008201C0312153DB261
:1014E0000CB401031215B1B40206C200C20FB20D52
:1014F000B40314200F0D1215B1C20CC20DC200D2DC
:101500000F8004D20CC20FB40419120999120327D8
:101510001209EF1202E440FB7FFFDFFE1202E440FB
:10152000F28008B405028003B40600754800121862
:10153000B5121B0D1200AC121C6F021CD07837794B
:1015400072121A69783B796E121A69200C15E53708
:10155000120764E553B4FF1802159E1218B585539F
:10156000528013E53B120764E553B4FF0302159E56
:101570001218B5855352E578857978F579E5785371
:1015800080CF4280D221120A1378727937121A69F9
:10159000786E793B121A69300E03120A1F22301D31
:1015A0000F12010E024D4F5554001203271215B1B0
:1015B00022200C06783B793780047837793B021A71
:1015C00069B40B11D21CE4785AF608B86EFB754D5D
:1015D00000C2098002C21C7F087837201C34300505
:1015E00031E55230200BC0E05380F04280D0E080E3
:1015F0000343800F75F009A42420F582758300123F
:1016000001C9F608A3DFF8121A2A4006121A42404E
:101610000122E552B40005901FBC8059B401059029
:101620001FC08051B40205901FC48049B4030590C7
:101630001FC88041B40405901FCC8039B4050590C3
:101640001FD08031B40605901FD48029B4070590BF
:101650001FD88021B40805901FDC8019B4090590BB
:101660001FE08011B40A05901FE48009B40B0590B7
:101670001FE88001227F047837C082C083121C5487
:10168000D083D0827F04783B021C54538900438965
:101690001143B808120A7C120B1FD28EC207755470
:1016A0000343A88FD288C209C20DC20FC21EC22234
:1016B000D20AD20CD22112187C2006030216F41290
:1016C00017F731581218361218621218731218517F
:1016D0009000071201C9A2E7920BA2E69204A2E5CC
:1016E000921DA2E492201217BE9000061201C9F5C5
:1016F00077021771754D03755632755528757680CA
:10170000757704D220C20BC204D21D755AFF755BD7
:10171000FF1217CE200503021771901FF4121793C2
:1017200090000B784312189F901FF01217939000AF
:101730000F784312189F901FEC12179390001378A4
:101740004312189F12184112185A12186B12184996
:10175000E5779000061201B1A20B92E7A20492E68F
:10176000A21D92E5A22092E49000071201B1121787
:10177000AE3020117552019007FF1201C9B4FF036A
:10178000021785F552B1C1121B0D121B98121C6F66
:10179000021CD07F047843C082C083121C54D083C3
:1017A000D082229000071201C9A2E7920B22E55ACB
:1017B0009000021201B1E55B9000030201B19000BC
:1017C000021201C9F55A9000031201C9F55BE55AEE
:1017D000A2E79213A2E69214A2E59215A2E4921651
:1017E000A2E39217A2E29218A2E19219A2E0921A41
:1017F000E55BA2E7921B2230051E784390000B2088
:101800001E10E5805430B4200390000FB4100390F4
:1018100000131218AA200508E47F047843F6DFFDC0
:1018200012182422C0E0D226121A59121C39121B97
:10183000C7C226D0E0229000041201C9F54DF54F31
:1018400022900004E54D0201B1900008E576020106
:10185000B19000081201C9F5762290000AE55602FF
:1018600001B190000A1201C9F55622900009E55510
:101870000201B19000091201C9F555229000001231
:1018800001C9B40104D2068010C20674011201B16C
:101890009000001201C9B40103D20522C205227FC3
:1018A00004E61201B108A3DFF8227F041201C9F691
:1018B00008A3DFF822201C1FC0E0E55275F009A440
:1018C00024207F087837F582758300E61201B1087D
:1018D000A3DFF8D0E08002113622754800201C0CEE
:1018E000201E09200A06300B03021999200A030260
:1018F00019C3754900754A00754B00754C00C0E06E
:10190000E54DB40005754C018042B40103754C02ED
:10191000B40203754C05B40303754C0AB404037593
:101920004C20B40503754C50B40603754B01B40745
:1019300003754B02B40803754B05B40903754B10CE
:10194000B40A03754A10B40B03754901D0E020E7CF
:1019500020FC121A1A794C121DE8201C10301D0DA3
:10196000121A425008121A1A794C121DF4DCE38044
:1019700020F404FC121A1A794C121DF4201C1030A9
:101980001D0D121A2A5008121A1A794C121DE8DC81
:10199000E3121B0D121C6F802AF4042576F57612D3
:1019A00000AC12010E020053706565643A00E576E2
:1019B000F41219C474071200C4E55AC2281219D5CA
:1019C0008556582275F06484F55A740AC5F084C4AB
:1019D00025F0F55B22E55AC0E0C4120149B4300598
:1019E0001201068005D2281200E2D0E0120149203F
:1019F0002808B430051201068005D2281200E2E55D
:101A00005BC0E0C4120149202808B4300512010669
:101A100080031200E2D0E002015E783A200C0278E6
:101A20003E227837200C02783B22511A7F04901F07
:101A300064E55223232403FEC3EE9396181EDFF9B8
:101A4000B322511A7F04901F90E55223232403FEF2
:101A5000C3EE9396181EDFF9227843800A78378008
:101A600006783B80025122793F7F04E6F70809DFC0
:101A7000FA22E552B40009301303021AEA021AF1FD
:101A8000B40109301403021AEA021AF1B40209304F
:101A90001503021AEA021AF1B40309301603021AF6
:101AA000EA021AF1B40409301703021AEA021AF121
:101AB000B40509301803021AEA021AF1B406093013
:101AC0001903021AEA021AF1B40709301A03021ABA
:101AD000EA021AF1B408028008B409028003B40AC9
:101AE00009301B03021AEA021AF178427946021DF4
:101AF000E878427946021DF400000170901AF87FE0
:101B000004785A121C547842795D021DE8C2AF3045
:101B100021051217F7C221301C085165121C2B0237
:101B20001B98300F1F51615172121C2B515D3023D5
:101B3000032004025172121C32301E0551FC121C8B
:101B400024021B98300D2351655172121C2BB20CCC
:101B500051653023032004025172121C32301E05DD
:101B600051FC121C24B20C021B9851653023032037
:101B700004025172121C32302303200406785A7971
:101B80002B5169301E0551FC121C24302303200404
:101B90000751655172121C2BC2AF201C26301E1C2F
:101BA00020861520A20530220780093022068000F9
:101BB0007836801578328011782E800D2086047852
:101BC000328006782E800278757E04E6121C421858
:101BD000DEF9901FF8E493121C42202609C2B5D208
:101BE000B5C2B5021BECC2B0D2B0C2B0D2AF22C2F5
:101BF000B7C2B5C2B0C2B67E057400121C42C2B5EF
:101C0000C2B0D2B5D2B0C2B5C2B018DEEC227E04EA
:101C10007400121C4218DEF87404121C42C2B0D2C6
:101C2000B0C2B022121E1179338013121E11792B0B
:101C3000800C121E11792F8005121E117972785AAC
:101C400041697D08135004D2B78002C2B7D2B6C230
:101C5000B6DDF122C0E0E493F6A308DFF9D0E0227C
:101C6000540F4430BF0705B4300274200200E22054
:101C70000D0D200F0A12010E0200412000800812F3
:101C8000010E02002020007837121CA6200D0D2026
:101C90000F0A12010E0240422000800812010E02BB
:101CA00040202000783B7F07BF0505742C1200E21E
:101CB000E6C0E0C491601FBF0006D0E09160800FD5
:101CC000BF0205742E1200E2D0E0916008DFD92235
:101CD00030090F740B200C02744B1200C4742A12CA
:101CE00000E2201C1F301E28C22330220B12010EDE
:101CF000020D46535200800912010E020D46534B4D
:101D000000021D5C12010E020D4D487A00021D5C9E
:101D1000E5805430B4001112010E020D43576E00DD
:101D20002023051217A3D223B4100D12010E020DA9
:101D300055534200C223C20BB4200D12010E020DF6
:101D40004C534200C223C20BB4301112010E020DDB
:101D5000435720002023051217A3D223300D2B74E4
:101D60004D1200C474531200E2200C1012010E0236
:101D700000540012010E02405200800E12010E02A9
:101D800000520012010E02405400300F18744D1220
:101D900000C474521200E212010E0200540012013B
:101DA0000E02405200200C0912010E02413E00803A
:101DB0000712010E02013E00201C1A30000A744D69
:101DC0001200C474431200E2744F1200C47431252F
:101DD0005212015E22227A04C39225E493A225378F
:101DE000D4F6A31819DAF2227A04C3E637D4F61827
:101DF00019DAF8227A04C3E69710D70730D60C9484
:101E000006800830D60294069460D3F61819DAE7F3
:101E100022785A7D14121E317A3F7E04121ED37826
:101E20005F7964121ECA121E60785B795A121ECA4C
:101E300022E4F608DDFC22901FF97E05785AE4932F
:101E4000F6A308DEF9785F7D0FD1317E057A5A124C
:101E50001ED37D05787AD1317863797E121F3822BE
:101E60007F2079637E0A121F21121E95121EA74041
:101E700011121EA1DFF3121E95121EA75003121E8F
:101E80008722121EBA80EA7F05785EC63400C61823
:101E90005002DFF722C378687E05C633C618DEFA23
:101EA000227E05785E80F37E057864797AC3E796B2
:101EB000600280050809DEF5D3227868797E7E0508
:101EC000C3C697C61819DEF9D3227A05E6F70809C2
:101ED000DAFA2278637968121F21121F01EAF8E604
:101EE000C0E0C478687963121F1379637868121FA1
:101EF00021121F01D0E078637968121F130ADED324
:101F0000227D04E675F00AA437F719E5F037F718D3
:101F1000DDF1227D04540FC336F6500418E480F836
:101F2000227D0589F0E4F719DDFCA9F02279687DAE
:101F30000FF1237E05D1D3227B01885A895B121FC2
:101F400048A85AA95B197B007C04E68BF0A437F7FC
:101F500019E5F037F75009E919C73400C740F9F916
:101F600018DCE72201740000034900000699000014
:101F70001009000013990000180670002099000055
:101F80002488000027990000499900004399000027
:101F9000020000000381000007210000101600006D
:101FA000143600001817000021460000250000002C
:101FB00029710000527100004601000001815000AB
:101FC00003710000070500001011600014270000D5
:101FD0001809600021060000249060002806000017
:101FE00050060000443000001000000009001500F9
:0E1FF000089985000900000000016000000053
:00000001FF
